S012000046696C653A204C6364322E61736D0A55
S113F0007EF0D6013CCE06868D0A38393CCE0343C9
S113F0108D02383909080926FB394F9701B71403C3
S113F020CEF036BDF04AE60008A600BDF07708BD74
S113F030F00C5A26F4390C30303020208000600067
S113F040C000103696018A01200536960184FE9789
S113F0500184F7B714033239C610BDF04A86802004
S113F06007C610BDF04A86C08D22BDF043A600BD80
S113F070F08C085A26F73984F097009601840F9A89
S113F08000970184F7B71403BDF0BF393C3684F010
S113F09097009601840F9A00970184F7B714038DA3
S113F0A01E324848484897009601840F9A009701F9
S113F0B084F7B714038D08CE000FBDF014383996C9
S113F0C0018A02970184F7B71403960184FD97011E
S113F0D084F7B71403398E8FFFBDF003BDF003BD71
S113F0E0F01ACEF0F1BDF058CEF101BDF0617EF022
S113F0F0EE20594F55204445534552564520412052
S113F100202020425245414B20544F444159202055
S104F11020DA
S105FFFEF0D637
S9030000FC
